S025000062696E2F64656D6F70726F675F6F6C696D65785F73746D3332683130332E7372656339
S3150800400000500020C1410008074200080942000884
S315080040100B4200080D4200080F420008000000008D
S315080040200000000000000000000000001142000827
S31508004030134200080000000015420008BD420008AF
S315080040401B4200081D4200081F42000821420008C2
S315080040502342000825420008274200082942000892
S315080040602B4200082D4200082F4200083142000862
S315080040703342000835420008374200083942000832
S315080040803B4200083D4200083F4200084142000802
S3150800409043420008454200084742000849420008D2
S315080040A04B4200084D4200084F42000851420008A2
S315080040B05342000855420008574200085942000872
S315080040C05B4200085D4200085F4200086142000842
S315080040D06342000865420008674200086942000812
S315080040E06B4200086D4200086F420008EE11AA559F
S315080040F010B5054C237833B9044B13B10448AFF314
S3150800410000800123237010BD680000200000000015
S31508004110C4450008084B10B51BB108490848AFF359
S3150800412000800848036803B910BD074B002BFBD075
S31508004130BDE81040184700BF000000006C000020D2
S31508004140C44500086800002000000000154B002B3D
S3150800415008BF134B9D46A3F5803A00218B460F46B0
S315080041601348144A121A00F017FA0F4B002B00D006
S3150800417098470E4B002B00D09847002000210400DA
S315080041800D000D48002802D00C48AFF3008000F05F
S31508004190DDF92000290000F01BF900F0C3F900BF83
S315080041A00000080000500020000000000000000089
S315080041B0680000208D0000200000000000000000BC
S315080041C006498D460649074A074B9A42BEBF51F82B
S315080041D0040B42F8040BF8E7044800470050002097
S315080041E0D045000800000020680000204D41000866
S315080041F01F49204A002301E041F8043B9142FBD3C2
S3150800420000F0E6F8FEE7FEE7FEE7FEE7FEE7FEE774
S31508004210FEE7FEE7FEE7FEE7FEE7FEE7FEE7FEE768
S31508004220FEE7FEE7FEE7FEE7FEE7FEE7FEE7FEE758
S31508004230FEE7FEE7FEE7FEE7FEE7FEE7FEE7FEE748
S31508004240FEE7FEE7FEE7FEE7FEE7FEE7FEE7FEE738
S31508004250FEE7FEE7FEE7FEE7FEE7FEE7FEE7FEE728
S31508004260FEE7FEE7FEE7FEE7FEE7FEE7FEE7FEE718
S31508004270680000208D000020014B1860704700BFC1
S315080042808400002008B5074B074A5A60F021074A00
S3150800429082F823100020986007221A60FFF7ECFFC7
S315080042A008BD00BF10E000E03F19010000ED00E086
S315080042B0014B1868704700BF84000020024A136843
S315080042C001331360704700BF8400002000B583B037
S315080042D000230193009303F1804303F504331A681E
S315080042E042F001021A605968364A0A405A601A684A
S315080042F022F0847222F480321A601A6822F480222C
S315080043001A605A6822F4FE025A604FF41F029A6035
S315080043101A6842F480321A602B4B1B6803F4003388
S315080043200093019B01330193009B23B9019A40F244
S31508004330DC539A42F0D1244B1B6813F4003F00D19A
S31508004340FEE7224B1A6842F010021A601A6822F039
S3150800435003021A601A6842F002021A60A3F5805333
S315080043605A685A605A6842F400525A605A6842F4C7
S3150800437080625A605A6822F47C125A605A6842F47B
S31508004380E8125A601A6842F080721A600E4B1B686F
S3150800439013F0007FFAD00C4B5A6822F003025A60D9
S315080043A05A6842F002025A60074B5B6803F00C0336
S315080043B0082BF9D100F074F8FFF764FF03B05DF835
S315080043C004FB00BF0000FFF8001002400020024076
S315080043D008B5FFF77BFF00F07DF8FCE721B1054B38
S315080043E09A69104398617047024A936923EA000064
S315080043F09061704700100240F0B4CB7803F00F02CA
S31508004400154613F0100F01D08D7815430B78E3B1DC
S315080044100668002316E001229A400C8832EA040452
S315080044200FD19C000F27A74026EA070605FA04F4D1
S315080044302643CC78282C01D1426102E0482C00D1D1
S3150800444002610133072BE6D906600B88FF2B1ED9BC
S315080044504668002318E003F108040122A2400C88EC
S3150800446032EA04040FD19C000F27A74026EA070664
S3150800447005FA04F42643CC78282C00D14261CC787E
S31508004480482C00D102610133072BE4D94660F0BC01
S31508004490704700BF0161704741617047FEE700BF82
S315080044A000B583B001211020FFF798FF4FF4805321
S315080044B0ADF8043003238DF8063010238DF8073045
S315080044C001A90348FFF798FF03B05DF804FB00BF96
S315080044D00010014010B5FFF7EBFE0F4B1B68C31A1F
S315080044E0B3F5FA7F16D304460C4B1B7843B9012261
S315080044F00A4B1A704FF480510948FFF7CDFF07E0C1
S315080045000022064B1A704FF480510548FFF7C2FF88
S31508004510014B1C6010BD00BF880000208C000020E5
S315080045200010014008B5074B044613B10021AFF34C
S315080045300080054B1868836A03B198472046FFF741
S31508004540ADFF00BF00000000C04500080E4B70B567
S315080045501E460E4C0025E41AA410A54204D056F8AF
S31508004560253098470135F8E700F01EF8084B094C46
S315080045701E46E41AA4100025A54204D056F8253094
S3150800458098470135F8E770BD6000002060000020FC
S31508004590600000206400002003460244934202D0D3
S315080045A003F8011BFAE77047F8B500BFF8BC08BC6A
S315080045B09E467047F8B500BFF8BC08BC9E467047D3
S30D080045C00000002000000000C5
S30D080045C884FBFF7F01000000DF
S315080045D000000000000000000000000000000000CD
S315080045E000000000000000000000000000000000BD
S315080045F000000000000000000000000000000000AD
S31508004600000000000000000000000000000000009C
S31508004610000000000000000000000000000000008C
S31508004620000000000000000000000000000000007C
S30D0800463015410008F1400008DD
S70508004000B2
